:0A00360000010202030304040505A3
:100F6F00C216C213D215C214120EB81213BD12112B
:100F7F0027121357750A0D750B0075120D75131285
:100F8F0075080D75091C75100D75114A75140D75C1
:100F9F00157890E680E030E70E85080C85090D8501
:100FAF00100E85110F800C85100C85110D85080E04
:100FBF0085090FD2E843D82090E668E04409F09005
:100FCF00E65CE0443DF0D2AF90E680E020E105D250
:100FDF00171212D0E58030E2107FF47E01120DBAA5
:100FEF0090E680E054F7F080031213FA538EF8C2A4
:100FFF0016E58020E2031213FA301405120762C2BD
:06100F001412040480EB42
:1013FA0090E680E04408F0E58030E2FB7FF47E016D
:0B140A00120DBA90E680E054F7F022CB
:1007620090E6B9E070030208351470030208D6243B
:10077200FE700302096224FB700302082F14700347
:1007820002082914700302081D14700302082324AE
:100792000560030209C990E6BBE024FE602C1460E8
:1007A2004724FD601614603124067065E50A90E660
:1007B200B3F0E50B90E6B4F00209D5E51290E6B38A
:1007C200F0E51390E6B4F00209D5E50C90E6B3F03B
:1007D200E50D90E6B4F00209D5E50E90E6B3F0E53A
:1007E2000F90E6B4F00209D590E6BAE0FF1212FFCC
:1007F200AA06A9077B01EA49600DEE90E6B3F0EF85
:1008020090E6B4F00209D590E6A0E04401F00209B6
:10081200D590E6A0E04401F00209D51214BF020906
:10082200D51214F20209D51214EA0209D51214AD36
:100832000209D590E6B8E0247F602B14603C2402C4
:1008420060030208CCA213E433FF25E0FFA215E403
:10085200334F90E740F0E4A3F090E68AF090E68B05
:100862007402F00209D5E490E740F0A3F090E68A22
:10087200F090E68B7402F00209D590E6BCE0547E5B
:10088200FF7E00E0D3948040067C007D0180047CE2
:10089200007D00EC4EFEED4F2436F58274003EF5ED
:1008A20083E493FF3395E0FEEF24A1FFEE34E68F5D
:1008B20082F583E0540190E740F0E4A3F090E68AE9
:1008C200F090E68B7402F00209D590E6A0E04401B4
:1008D200F00209D590E6B8E024FE601D2402600310
:1008E2000209D590E6BAE0B40105C2130209D59017
:1008F200E6A0E04401F00209D590E6BAE070589013
:10090200E6BCE0547EFF7E00E0D3948040067C008B
:100912007D0180047C007D00EC4EFEED4F2436F517
:100922008274003EF583E493FF3395E0FEEF24A149
:10093200FFEE34E68F82F583E054FEF090E6BCE0F1
:100942005480FF131313541FFFE0540F2F90E683BC
:10095200F0E04420F0807C90E6A0E04401F0807357
:1009620090E6B8E024FE60202402706790E6BAE0C8
:10097200B40104D213805C90E6BAE0640260549041
:10098200E6A0E04401F0804B90E6BCE0547EFF7E9E
:1009920000E0D3948040067C007D0180047C007DD1
:1009A20000EC4EFEED4F2436F58274003EF583E4F2
:1009B20093FF3395E0FEEF24A1FFEE34E68F82F53C
:1009C20083E04401F0800C120056500790E6A0E04C
:0A09D2004401F090E6A0E04480F03C
:0109DC0022F8
:0300330002001FA9
:04001F0053D8EF3291
:1012D00030170990E680E0440AF0800790E680E04D
:1012E0004408F07FDC7E05120DBA90E65D74FFF0D5
:0F12F00090E65FF05391EF90E680E054F7F02224
:100DBA008E4C8F4D90E600E054187012E54D2401D8
:100DCA00FFE4354CC313F54CEF13F54D801590E64F
:100DDA0000E05418FFBF100BE54D25E0F54DE54C3A
:100DEA0033F54CE54D154DAE4C7002154C4E600571
:060DFA001214D180EE226C
:0212FF00A9073D
:10130100AE14AF158F828E83A3E064037017AD0115
:1013110019ED7001228F828E83E07C002FFDEC3E5F
:09132100FEAF0580DF7E007F00B5
:01132A0022A0
:1014D1007400F58690FDA57C05A3E582458370F92E
:0114E10022E8
:03004300020E00AA
:03005300020E009A
:100E0000021415000214710002145B0002142D007C
:100E10000211CE00021191000200420002004A00BD
:100E200002005200020CFF0002150A0002150B001E
:100E300002150C0002150D0002150E0002150F0020
:100E40000215100002004A000215110002151200DE
:100E500002151300021514000215150002151600E4
:100E60000215170002004A0002004A0002004A0070
:100E7000021518000215190002151A0002151B00B0
:100E800002151C0002151D0002151E0002151F0090
:100E90000215200002152100021522000215230070
:100EA0000215240002152500021526000215270050
:080EB0000215280002152900BB
:100D0000120100020000004004230402000001025E
:100D100000010A06000200000040010009022E0046
:100D2000010100C0320904000004FF0000000705B3
:100D30000202000200070504020002000705860205
:100D40000002000705880200020009022E000101CE
:100D500000C0320904000004FF0000000705020281
:100D6000400000070504024000000705860240001D
:100D70000007058802400000040309042203500014
:100D800069006E006E00610063006C006500200069
:100D9000530079007300740065006D0073001A033E
:100DA0004D006F0076006900650042006F0078001A
:0A0DB000200055005300420000002F
:060AE500011800011900D8
:10137B00759850758920758780758DD9758BD9D2E5
:10138B008E438E10D2ACD2BCD2AFC2997E007F00FE
:01139B00222F
:10135700E4FFFE7E50901A87E4F0A3DEFC7E007F58
:1013670050E4F516F517F51CF51DF51AF51B1213C4
:031377007BFEFFFB
:01137A002250
:03002300020BE9E4
:100BE900C0E0C0F0C083C082C0D075D000C000C0D2
:0D0BF90001C002C003C004C005C006C00753
:100C0600309923C299C3E51D9517E51C9516501614
:100C16007487251DF582E4341AF583E0F599051DE0
:100C2600E51D7002051C309866C298AF99BFAA06EA
:100C3600751A00751B00C3E51B9450E51A94005005
:100C46001674D9251BF582741A351AF583EFF0054B
:100C56001BE51B7002051ABFAA0AE51B14F51875D9
:100C66002AAA802B74D8251BF582741A351AF583A7
:100C7600E0B52A0AE51B14F5191212A0801174D8E2
:0F0C8600251BF582741A351AF583E0252AF52A05
:100C9500D007D006D005D004D003D002D001D000B3
:0B0CA500D0D0D082D083D0F0D0E0325D
:1012A000901ADAE064447027901AE2E0FFB4010378
:1012B000C20422EF7019D204901AE3E0FFB40104D3
:1012C000C2048005EF7002D204901AE6E0F53D22D8
:100AEB0060801A0001010105253D0107000400008B
:100AFB0007010000FBF3E7E7E7F7F7FF0009121226
:100B0B00C832123F01010101253D0107000002001F
:100B1B0001050000FBF3F7D7D7F7F7FF090912120E
:100B2B00C8F2363F01010105250101070000000055
:100B3B0001020000FBF3F7E7E7E7F7FF00091212EA
:100B4B00C82D123F01010101052E01070000000213
:100B5B0002030000FBF3F7F7D7D7D7FF09091212EF
:0E0B6B0000C8363F471A80800000FF06E411E4
:1011270090E60174CEF090E6F574FFF0901A80E037
:1011370090E6F3F0901A81E090E6C3F0901A82E00F
:1011470090E6C1F0901A83E090E6C2F0901A85E02D
:1011570090E6C0F0901A86E090E6F4F075AF077459
:101167001AF59A7400F59B759DE4E4F59EFF90E6E9
:101177007BE090E67CF00FBF80F4000000E490E68F
:09118700C4F000000090E6C5F080
:01119000223C
:100CB0008E4C8F4DE4F527F526F525F524E5BB2070
:100CC000E72F7FF07E497D027C00AB27AA26A9256D
:100CD000A824C31210F07002C322E5272401F527CF
:100CE000E43526F526E43525F525E43524F524807C
:0F0CF000CCE54C90E6F0F090E6F1E54DF0D32224
:04132B00AD07AC0658
:10132F00E4FFE5BB30E7FB90E6F1E0FFE5BB30E71C
:10133F00FB90E6F0E0FE90E6F2E0FBEEEBFF8D8235
:07134F008C83EEF0A3EFF028
:011356002274
:0814E200E5BB30E7FB8FBB22E4
:10148700AC0600000090E6D0ECF000000090E6D13A
:03149700EFF02251
:0B002600E5BB30E7FBEF4404F5BB2214
:10149A00AC0600000090E6D0ECF000000090E6D127
:0314AA00EFF0223E
:100B790060281AEF000000000000000000000000DB
:100B8900000000000000000000000000000000005C
:100B9900000000000000000000000000C106C100C4
:100BA900C112C18AC18E042400000000C10D0231A6
:100BB9000100022B0040C102C109023B0000C1072C
:100BC900C10BC10FC111C101044100030D4004371C
:0F0BD90000000000C104C10C013D00C110C105A6
:040046005380F722CA
:04004E0043800822C1
:041502005380EF2201
:0415060043801022EC
:0A1445007B017A1A79ED7F0C7E001E
:0C144F0090D000EFF0AE02AF0102132BB2
:10139C00E4F53FF54074D92540F582E4341AF58321
:1013AC00E4F00540E5407002053F6414453F70E5EC
:0113BC00220E
:100EB80090E600E054E74410F01214FA75B2FBE42F
:100EC800F5B375B4FFF5B5F5B6F5805380FC7F0131
:100ED800FE120DBA4380035380FD75A01012004E18
:100EE80012150690E61074A0F090E611F0000000CC
:100EF80090E61274A2F000000090E61374A0F000CF
:100F0800000090E61474E2F000000090E61574E02A
:100F1800F000000090E6917480F0000000F00000FE
:100F28000090E695F0000000F000000090E604F064
:100F38000000007406F0000000E4F090E680E03065
:100F4800E710753101753200752B00752C40D208F9
:100F5800800E753100753220752B02752C00C20881
:070F680012139C43AF0122AC
:1013BD0053A0DF53807F7F017E00120DBA43A02022
:1013CD007F017E00120DBA4380807F017E00020DE9
:0113DD00BA55
:1004040030066BE5AA20E06690E690E0FE90E69167
:10041400E07C002400F530EC3EF52FE4F53FF54098
:10042400C3E5409530E53F952F503D74002540F5D8
:100434008274F0353FF583E0752800F529740125B1
:1004440040F58274F0353FF583E0FEE4EE42283057
:100454000B09AF29AE28120CB0920B74022540F59B
:1004640040E4353FF53F80B890E6917480F0200079
:100474000302068DE5AA30E50302068D30106612EC
:100484001445901AEEE030E1367B017A1A79D77F71
:10049400067E0012144F901AD7E0B4EE1DA3E0B408
:1004A400FF18C200C209C210C202C201D20AC207A6
:1004B400E4F53BF53CC20512004E12144580C330EE
:1004C4000203300A0630021D30011AC200C209C2FA
:1004D40010C202C201D20AC207E4F53BF53CC205D0
:1004E400C20B12004E20090302068D121445E4F5D6
:1004F40027F526F525F524901AEDE0A320E459AF5D
:1005040044AE43AD42AC41AB27AA26A925A824C3D7
:100514001210F05043200140121445E5272401F540
:1005240027E43526F526E43525F525E43524F52498
:10053400AF44AE43AD42AC41AB27AA26A925F8C3CC
:100544001210F070B21215027FF47E01120DBA126D
:100554001506D201C20B809FE5AA30E50302068D81
:10056400C3E53C952CE53B952B400302068D200109
:100574001A300A1790D0007480F0300A32AF32AECD
:100584003112149A7F021200268024E4F53FF540CC
:1005940074002540F58274F8353FF58374FFF00547
:1005A40040E5407002053FB400E6E53FB402E1E4F3
:1005B400F527F526F525F524300A65E5BB20E76027
:1005C4007FA07E867D017C00AB27AA26A925A824CE
:1005D400C31210F07033C20A200202C20B90E6F577
:1005E40074FFF0E4F53FF54074002540F58274F89B
:1005F400353FF58374FFF00540E5407002053FB4D4
:1006040000E6E53FB402E18017E5272401F527E47D
:100614003526F526E43525F525E43524F52480989A
:1006240030081300000090E6987402F0000000E423
:1006340090E699F08011000000E490E698F0000044
:100644000090E6997440F030071400000090E6042E
:100654007480F00000007406F0000000E4F0053C33
:10066400E53C7002053BB52C20E53BB52B1BE4F5BE
:100674003BF53CC209300204D207D209E58030E3DD
:1006840005120046800312004E201203020761E5A2
:10069400AA30E203020761121445901AEEE030E139
:1006A400127B017A1A79D77F067E0012144F121436
:1006B4004580E7901AEDE0A320E41E901AEEE030A6
:1006C400E1127B017A1A79D77F067E0012144F1249
:1006D400144580E712144580DA90D0007480F0301D
:1006E4000E11E490E695F0AF32AE311214877F011B
:1006F4001214E2E4F527F526F525F524300E3CE541
:10070400BB20E7377FA07E867D017C00AB27AA262D
:10071400A925A824C31210F0400AC20E90E6F5746D
:10072400FFF08017E5272401F527E43526F526E4B4
:100734003525F525E43524F52480C1053CE53C70D8
:1007440002053BB52C17E53BB52B12E58030E405DB
:0E0754001215028003121506E4F53BF53C2257
:02003100D322D8
:02004000D322C9
:0814EA0090E6BAE0F53ED322C2
:1014AD0090E740E53EF0E490E68AF090E68B04F09C
:0214BD00D32238
:0814F20090E6BAE0F523D322D5
:1014BF0090E740E523F0E490E68AF090E68B04F0A5
:0214CF00D32226
:1000560090E6B9E012110103E6A402AFA802CEA908
:10006600027DAA01F9AB0221AD024FAE02FBBA0333
:1000760022C400ACC50345CB0088D0009AD100004D
:10008600040090E604E0F54B434B80000000E54B8E
:10009600F002040290E604E0F54B534B7F000000AB
:1000A600E54BF0020402E490E68AF000000090E6D8
:1000B6008BF090E6A0E020E1F990E740E012110114
:1000C6000195A600E8A701B3AC01A8B100EEB20104
:1000D60001B30151B40184BC01CDC901DFCD0000DB
:1000E60001F71213BD02040290E741E0B40107D202
:1000F60006D20B020402C20602040290E741E0B4F3
:10010600012A90D0007408F07F017E00120CB0D254
:100116000AD200C20FC21175444075430D754203E1
:10012600754100E4F52FF530D205801790D00074A4
:1001360008F0E4FFFE120CB0D202D210D207D209A8
:1001460012004EE490E6E3F002040290E741E0B4C8
:10015600011390D0007408F07F017E00120CB0D21B
:100166000ED212801190D0007408F0E4FFFE120C3B
:10017600B0121506C212E490E6DBF002040290E724
:1001860041E0B40105D209020402C2090204029048
:10019600E741E0B401064380400204025380BF02F7
:1001A600040290E741E090D000F002040290E7419B
:1001B600E0752800F529A3E0FEE4EE4228AF29AE5B
:1001C60028120CB002040290E741E060065380FD5D
:1001D60002040243800202040290E741E0600953F0
:1001E60080DF4380400204024380205380BF020424
:1001F60002D3227E1A7FED12132B901AEDE090E7C0
:1002060040F0901AEEE090E741F0E490E68AF000C4
:10021600000090E68B7402F002040290D000740C89
:10022600F07E1A7FED12132B901AEDE090E740F066
:10023600901AEEE090E741F0E490E68AF0000000C4
:1002460090E68B7402F002040290D0007406F07EF1
:100256001A7FED12132B901AEDE090E740F0901AFA
:10026600EEE090E741F0E490E68AF000000090E6C8
:100276008B7402F0020402E490E68AF0000000901B
:10028600E68BF090E6A0E020E1F990E740E0752DDE
:1002960000F52EA3E0753500F536AF2EFD7AE77B27
:1002A600421213DE9203020402E490E68AF0000092
:1002B6000090E68BF090E6A0E020E1F990E740E0C0
:1002C600753300F534020402AF2EAD347AE77B4075
:1002D6001200035011E490E68AF000000090E68BCD
:1002E600E534F0020402E490E68AF000000090E6AD
:1002F6008BF002040290E680E030E70890E7407455
:1003060001F08005E490E740F0000000E490E68A02
:10031600F000000090E68B04F0020402300B089017
:10032600E7407401F08005E490E740F0000000E447
:1003360090E68AF000000090E68B04F00204027B4F
:10034600017A1A79ED7F267E0012144F901AEDE09D
:1003560090E740F0901AEEE090E741F07B017A1AC0
:1003660079ED7F247E0012144F901AEDE090E7425B
:10037600F0901AEEE090E743F07B017A1A79ED7F70
:10038600227E0012144F901AEDE090E744F0901A86
:10039600EEE090E745F07B017A1A79ED7F207E004A
:1003A60012144F901AEDE090E746F0901AEEE090A6
:1003B600E747F07B017A1A79ED7F287E0012144F09
:1003C600901AEDE090E748F0901AEEE090E749F0D9
:1003D600E490E68AF000000090E68B740AF0801C38
:1003E600A205E43390E740F0000000E490E68AF0CE
:0D03F60000000090E68B04F08002D322C3CB
:0104030022D6
:10141500C0E0C083C082D2145391EF90E65D7401A1
:08142500F0D082D083D0E03248
:10145B00C0E0C083C0825391EF90E65D7404F0D07E
:06146B0082D083D0E032C4
:10147100C0E0C083C0825391EF90E65D7402F0D06A
:0614810082D083D0E032AE
:1011CE00C0E0C083C08285100C85110D850D82850F
:1011DE000C83A37402F085080E85090F850F828596
:1011EE000E83A37407F05391EF90E65D7410F0D068
:0611FE0082D083D0E03234
:10142D00C0E0C083C082D2165391EF90E65D740880
:08143D00F0D082D083D0E03230
:10119100C0E0C083C08290E680E030E72085080C83
:1011A10085090D850D82850C83A37402F085100ECF
:1011B10085110F850F82850E83A37407F05391EF7C
:0D11C10090E65D7420F0D082D083D0E03243
:01004200328B
:01004A003283
:01005200327B
:010CFF0032C2
:01150A0032AE
:01150B0032AD
:01150C0032AC
:01150D0032AB
:01150E0032AA
:01150F0032A9
:0115100032A8
:0115110032A7
:0115120032A6
:0115130032A5
:0115140032A4
:0115150032A3
:0115160032A2
:0115170032A1
:0115180032A0
:01151900329F
:01151A00329E
:01151B00329D
:01151C00329C
:01151D00329B
:01151E00329A
:01151F003299
:011520003298
:011521003297
:011522003296
:011523003295
:011524003294
:011525003293
:011526003292
:011527003291
:011528003290
:01152900328F
:0814FA00E4F54AD2E9D2AF2269
:1012040090E678E020E6F9C2E990E678E04480F0E0
:10121400EF25E090E679F090E678E030E0F990E6AA
:1012240078E04440F090E678E020E6F990E678E053
:0612340030E1D6D2E922F0
:10126E00A90790E678E020E6F9E54A702390E67843
:10127E00E04480F0E925E090E679F08D45AF03A9D2
:10128E00077546018A478948E4F549754A01D32214
:02129E00C32269
:10123A00A90790E678E020E6F9E54A702590E67875
:10124A00E04480F0E925E0440190E679F08D45AF6D
:10125A0003A9077546018A478948E4F549754A038F
:04126A00D322C322A6
:03004B000209DDCA
:1009DD00C0E0C083C082C085C084C086758600C05B
:1009ED00D075D000C000C001C002C003C006C00752
:1009FD0090E678E030E206754A06020AC790E6787E
:100A0D00E020E10CE54A64026006754A07020AC758
:100A1D00E54A24FE605F14603624FE7003020AB8B6
:100A2D0024FC7003020AC424086003020AC7AB4603
:100A3D00AA47A948AF4905498F827583001210A1B5
:100A4D0090E679F0E54965457070754A05806B90C3
:100A5D00E679E0AB46AA47A948AE498E8275830078
:100A6D001210CE754A02E5456401704E90E678E0AD
:100A7D004420F08045E54524FEB5490790E678E031
:100A8D004420F0E54514B5490A90E678E04440F07D
:100A9D00754A0090E679E0AB46AA47A948AE498E63
:100AAD00827583001210CE0549800F90E678E044E0
:100ABD0040F0754A008003754A005391DFD007D08E
:100ACD0006D003D002D001D000D0D0D086D084D0B3
:080ADD0085D082D083D0E03205
:1000030012123AE54A24FA600E146006240770F3CC
:0C001300D322E4F54AD322E4F54AD322BC
:1013DE0012126EE54A24FA600E146006240770F3AA
:0C13EE00D322E4F54AD322E4F54AD322CE
:03000000021015D6
:0C101500787FE4F6D8FD75814D02105C78
:1010A100BB010CE58229F582E5833AF583E0225004
:1010B10006E92582F8E622BBFE06E92582F8E2224E
:0D10C100E58229F582E5833AF583E4932268
:1010CE00F8BB010DE58229F582E5833AF583E8F058
:1010DE00225006E92582C8F622BBFE05E92582C804
:0210EE00F222EC
:1010F000EB9FF5F0EA9E42F0E99D42F0E89C45F056
:0111000022CC
:10110100D083D082F8E4937012740193700DA3A37D
:1011110093F8740193F5828883E473740293686091
:06112100EFA3A3A380DF91
:10102100020F6FE493A3F8E493A34003F68001F267
:1010310008DFF48029E493A3F85407240CC8C333D0
:10104100C4540F4420C8834004F456800146F6DF9F
:10105100E4800B0102040810204080900AE5E47E40
:10106100019360BCA3FF543F30E509541FFEE49394
:10107100A360010ECF54C025E060A840B8E493A35B
:10108100FAE493A3F8E493A3C8C582C8CAC583CA86
:10109100F0A3C8C582C8CAC583CADFE9DEE780BE3E
:010BE800000C
:00000001FF
